:020000040800F2
:10000000B01D00209D0100085B1E0008271D000890
:10001000591E0008A9020008051F00080000000082
:10002000000000000000000000000000751E000835
:10003000F1060008000000005D1E0008771E0008A1
:10004000B7010008B7010008B7010008B7010008B0
:10005000B7010008B7010008B7010008B7010008A0
:10006000B7010008B7010008B7010008B701000890
:10007000B7010008B7010008B7010008B701000880
:10008000B7010008B7010008B7010008B701000870
:10009000F91E0008B7010008B7010008B701000801
:1000A000B7010008B7010008B7010008B701000850
:1000B000B7010008B7010008B7010008B701000840
:1000C000B7010008B7010008B7010008B701000830
:1000D000B7010008B7010008B7010008B701000820
:1000E000B7010008B7010008B701000800000000D0
:1000F0000000000000000000000000000000000000
:10010000000000000000000000000000B70100082F
:10011000B7010008B7010008B7010008000000009F
:10012000B7010008B7010008B7010008B7010008CF
:10013000B7010008000000000000000000000000FF
:10014000B7010008B701000800000000000000002F
:10015000000000000000000000000000000000009F
:100160000000000000000000B7010008B70100080F
:10017000B7010008000000000000000000000000BF
:1001800000000000B7010008DFF80CD000F07AF89A
:10019000004800474D200008B01D00200648804759
:1001A00006480047FEE7FEE7FEE7FEE7FEE7FEE75C
:1001B000FEE7FEE7FEE7FEE7E91E0008890100080A
:1001C0002DE9F05F0546002092469B46884606468C
:1001D000814640241BE0284641464746224600F01F
:1001E00020F853465A46C01A914110D3114618467A
:1001F000224600F038F82D1A67EB01084F462246D8
:100200000120002100F02FF817EB00094E41201EBD
:10021000A4F10104DFDC484631462A464346BDE8E6
:10022000F09F202A04DB203A21FA02F000217047D7
:1002300021FA02F3D040C2F120029140084319464E
:100240007047D2B201E000F8012B491EFBD2704783
:100250000022F6E710B513460A4604461946FFF792
:10026000F0FF204610BD202A04DB203A00FA02F1FC
:10027000002070479140C2F1200320FA03F3194394
:1002800090407047064C074D06E0E06840F00103DF
:1002900094E8070098471034AC42F6D3FFF778FF94
:1002A000EC2700080C280008FEE710B54FF4D872C0
:1002B000036802EB01129B5803F00404436B9C603B
:1002C000436B002C57D00468A458E4085C600368B2
:1002D0009A58436B02F00202DA604FF4DA72036854
:1002E00002EB01129B58446B03F00F032361036878
:1002F0009A58436BC2F30722DA614FF4DC72036849
:1003000002EB01129B58446B237503689B58446BA6
:100310001B0A637503689B58446B1B0CA375036829
:100320009A58436B120EDA754FF4DE72036802EBD3
:1003300001129B58446B237603689B58446B1B0A3D
:10034000637603689B58446B1B0CA37603689A582A
:10035000436B120EDA7699B101680A6942F0200205
:100360000A6101684A6922F010024A6190F8391066
:10037000222910D014E00468A458640D1C60A6E77C
:100380000168CA6842F02002CA6001684A6922F026
:1003900002024A61EAE701684A6922F40F424A61AF
:1003A00090F83910322906D0012180F8391000F078
:1003B000B3FC002010BD122180F83910F7E70000CF
:1003C00030B500221BE00F4B85885C6B02F11403F3
:1003D000E35CC468635583885B1C9CB2848043885B
:1003E0009C4201D3002484800489641CA4B204814B
:1003F0009C4202D9038101238372521CD2B28A42E9
:10040000E1D330BDA400002010B501684A6922F094
:1004100001024A6190F83910122904D101684A6931
:1004200022F40F424A6190F83910322906D0012196
:1004300080F8391000F06AFD002010BD222180F8FC
:100440003910F7E72DE9F14F82B0029800890B28A7
:100450005ED30021029801F0E9FD044601210298D3
:1004600001F0E4FD552C01D1AA2806D0029803B072
:100470000121BDE8F04F01F0A5BD0221029801F075
:10048000D5FD04460321029801F0D0FD0546052163
:10049000029801F0CBFD06460421029801F0C6FD4A
:1004A00006EB00201FFA80FA162C06D0029803B043
:1004B0000121BDE8F04F01F085BD0298018905F1E9
:1004C00009000190814223D3DFF87881552088F814
:1004D0000000AA2088F80100072088F802005120B7
:1004E00088F8030005F10801029801F09FFD01273B
:1004F000DFF85491554EF0280CD00121029801F0FC
:1005000061FD89F800704CF20230B080F020B070CC
:10051000BDE8FE8F291D029801F088FD0406691DC3
:10052000029801F083FD04EB0044A91D029801F03C
:100530007DFD04EB0024E91D029801F077FD2044C5
:100540000090022405F1040B08E02146029801F016
:100550006DFD08EB04018870641CA4B25C45F4D303
:10056000A91D384800F078F8009981420DD089F82B
:1005700000704CF20230B080F120B070DDE9011063
:1005800003B0BDE8F04F01F01DBDDDE9011001F041
:1005900019FD0024A9F80240AAF5145ABAF1050A77
:1005A0004BD0AAF5F84ABAF1060A4FF480650ED08E
:1005B000AAF5007ABAF17A0A22D0BAF17C0F34D0C7
:1005C000029803B00121BDE8F04F01F0FBBCB07808
:1005D00001289DD0B77089F800704CF20240B080BD
:1005E000D8F80F00F0601A4800F08AF80020194986
:1005F0000C54401C80B2A842FAD3A9F8044087E703
:100600000220B0700F480D30B06098F8090098F8DB
:100610000A1000EB012080B2F080A84200D3F480E1
:100620004CF20220B080377072E70320B07089F876
:1006300000704CF20250B0806AE70520B07089F873
:10064000007065E7F804002004000020E4000020AA
:1006500000300008F800002070B506464FF0FF306B
:100660000023094D0DE0F25C50400022040E55F8C5
:10067000244000026040521C92B2042AF6D35B1C54
:100680009BB28B42EFD370BDBC230008F0B58BB09A
:10069000002406940794012508954EF2200001904D
:1006A00002944EF2E01703974FF6FF7604960594F6
:1006B000099501A90D4800F0EDF808B100F019F80E
:1006C0000695079408954FF46040019002940397B3
:1006D00004960594099501A9044800F0DBF8002868
:1006E00001D000F006F80BB0F0BD0000A40000201F
:1006F0007047012484F3138800F0CAFEFAE7000073
:100700007FB5044600260396002500F0B5FC0B4893
:1007100084420AD2401C001BC00A00960194029039
:1007200003A9684600F006FC054600F055FC15B12B
:10073000012004B070BD0020FBE70000FFDF0108CE
:1007400010B500F099FC03493420C860BDE81040A2
:1007500000F042BC002002402DE9F04105460E4663
:100760001746002400F088FCDFF83C8013E056F8C0
:10077000242000232946022000F038FC10B1032079
:10078000BDE8F08156F824102868884201D0022084
:10079000F6E72D1D641CBC4201D24545E7D900F0A7
:1007A0001BFC0020ECE70000FBDF010806490020ED
:1007B000C8610648016941F004010161016941F025
:1007C0004001016170470000900D002000200240B0
:1007D000064A0021D16106490A6942F002020A6113
:1007E0004861086940F0400008617047900D0020A2
:1007F00000200240044B0022DA61044A136943F0EE
:100800000103136101807047900D00200020024019
:1008100000200A4AD168CB06094904D5C86940F0CE
:100820000200C8611020D3685B0705D5CB6943F08F
:100830000103CB6140F00400D0607047002002400B
:10084000900D002070B5044600F07AFD0546104E6C
:1008500009E0601C07D024B100F072FD401BA042EB
:1008600001D9032070BDF068C007F2D1F06880069E
:1008700001D52020F060F068C00602D4F06840077F
:1008800003D5FFF7C5FF012070BD002070BD00003B
:1008900000200240F0B50B7D012404FA03F2036846
:1008A000D3F800524E6A25F47C5504EB0624254308
:1008B000C3F800520368D3F81C429443C3F81C42A7
:1008C0004FF41075CB692E1D002B17D10368D3F898
:1008D0000C429443C3F80C428C894B684F6964F313
:1008E0001F43046805EBC707E3510C890B684F6988
:1008F00064F31F43046806EBC707E351CB69012B80
:1009000017D10368D3F80C421443C3F80C420C8887
:100910004B684F6964F31F43046805EBC7056351D7
:100920000C89CB684D6964F31F43046806EBC50569
:1009300063518B698BB10368D3F804421443C3F845
:1009400004420B6983B10368D3F814421443C3F81B
:100950001442096A01290ED013E00368D3F8044257
:100960009443C3F80442ECE70368D3F81442944379
:10097000C3F81442EDE70168D1F81C321343C1F803
:100980001C320068D0F8001221F00101C0F80012FA
:100990000020F0BD10B50446002C0AD0022084F8D7
:1009A0003900204600F052F9002038346070207081
:1009B00010BD012010BD0068416941F00201416194
:1009C0007047000010B5044620684169C943C90753
:1009D0000ED182685049914307D082684F499143B4
:1009E00003D081684E48884302D12046FFF70CFDB2
:1009F00020684169C943890706D4C068800703D0CD
:100A000000212046FFF751FC20684169C943C9060F
:100A100006D40069800703D001212046FFF745FC7A
:100A200020688169C9070BD04169C943C90507D44A
:100A30004169C943090403D4E16B41F00101E16359
:100A4000816989070BD54169C943890507D4416983
:100A5000C943090403D4E16B41F00201E1638169F8
:100A600049070BD54169C943490507D44169C943C1
:100A7000090403D4E16B41F00401E163816911F0E1
:100A8000700F3AD04169C943090536D44169C94359
:100A9000090432D4816901F0700140291BD006DCC1
:100AA000102909D020290CD0302922D10EE050295C
:100AB00016D060291DD118E0E16B41F00801E16317
:100AC00017E0E16B41F01001E16312E0E16B41F0EE
:100AD0002001E1630DE0E16B41F04001E16308E0DA
:100AE000E16B41F08001E16303E0E16B41F480716F
:100AF000E163816921F070018161E06B00280AD017
:100B00002068416841F004014160012084F8390007
:100B10002046FFF750FF10BD03000004000300084B
:100B2000000003102DE9F047044600270025002CA3
:100B300004D094F83900A84618B107E00120BDE8B8
:100B4000F08784F83880204600F09CF8022084F872
:100B500039002068016821F0020101602068016805
:100B600041F00101016000F0EBFB06464FF0030984
:100B70000AE000F0E5FB801B0A2805D984F83990CB
:100B800084F838800320DAE720684068C007F0D096
:100B900020684168C9074BD0A169012901D145F0FE
:100BA0008005E169012901D145F04005216A01294B
:100BB00001D145F02005616A012901D145F01005F8
:100BC000A16A012901D145F00805E16A012901D195
:100BD00045F00405016821F0FC0129430160D4E9D6
:100BE00002010843D4E90412114308436168491E15
:100BF00008432168C8612068016821F00101016093
:100C000000F09EFB05460AE000F09AFB401B0A2814
:100C100005D984F8399084F8388003208FE720685C
:100C20004068C007F0D120684068C00700D10127A4
:100C3000012F04D0042084F8390001207FE7C4F894
:100C40003C80012084F83900002078E710B5006866
:100C5000094988420ED10948C16921F00071C1617A
:100C60004FF44071064800F01BFABDE81040142014
:100C700000F0BEBB10BD0000006400400010024048
:100C80000004004810B586B00446142101A8FFF7FF
:100C9000DFFA1D492068884234D11C48C16941F0FF
:100CA0000071C161C16901F000710091416941F4B5
:100CB00080214161406900F4802000904FF4407031
:100CC000019012200290002003900320049009203C
:100CD000059001A90E4800F05BFA0022114614208D
:100CE00000F0A4FB142000F094FB0A4800F140043B
:100CF00020631C306063FFF7C9FC2068416941F044
:100D00000201416106B010BD0064004000100240C5
:100D1000000400486400002010B5406B0D4C816851
:100D2000002910D1016971B10068A0F5E062513A63
:100D300003D1C9B20848FFF743FB2068416941F07D
:100D40000201416110BD2068416941F00201416129
:100D500010BD0000A4000020440000202DE9F05F39
:100D600004460E46042594F83800012810D04FF0B0
:100D7000010884F8388094F8390022280BD012201A
:100D800084F8390021688868400108D500250FE003
:100D90000220BDE8F09F322084F83900F2E788682D
:100DA000000101D5012503E08868C00000D50225B7
:100DB0000027042D78D04FF4C07000EB05100A58BE
:100DC00002F001020A50216B8A68EAB3236853F8E3
:100DD00000C04CEA020CCA68496842EAC1014CEA08
:100DE000010C43F800C0216B0A7C02F00F020A617B
:100DF0004FF4C271226801EB0511535823F00F0321
:100E0000535022685358D4F830C0DCF810C043EA7D
:100E10000C035350216B0A7DCB7D42EA03628B7D2C
:100E2000497D1B0443EA01210A434FF4C47321683E
:100E300003EB0513CA50216B0A7ECB7E42EA0362A4
:100E40008B7E497E1B0400E015E043EA01210A4342
:100E50004FF4C673216803EB0513CA5021680A5882
:100E600042F001020A5000F06BFA8146DFF890A0D0
:100E7000DFF890B019E022681358D1F80CC0098847
:100E800043EA0C0343EA41511150ACE7701C0CD00B
:100E90002EB100F055FAA0EB0900B04205D90320AD
:100EA00038346070277074E723E085B1012D14D0C9
:100EB0002068816814488843E8D194F839003228C2
:100EC00011D084F8398084F83870002061E72068F8
:100ED00080683AEA0000F0D0D8E7206880683BEAF2
:100EE0000000EAD0D2E7222084F8390084F8387074
:100EF000E9E70420383460702770012049E70000DA
:100F00000300000400030008000003107047000005
:100F100070B5044600F014FA0546601C02D004487F
:100F20000078044400F00CFA401BA042FAD370BDD4
:100F3000540000202DE9F04705460F464FF0010A06
:100F4000DFF88C8098F8180001280DD0012088F86F
:100F5000180028681F4E4CF25039012807D0484627
:100F6000FFF770FC90B12EE00220BDE8F087484604
:100F7000FFF768FC38BBFFF719FC4846FFF762FC37
:100F80008246306920F0040030611CE04FF0FF30F1
:100F900038606C6811E02046FFF71AFC4846FFF7FE
:100FA00051FC8246306920F0020030615FEA0A009D
:100FB00001D03C6007E004F50064D5E9010100EBD5
:100FC000C120A042E7D8002088F818005046CCE79E
:100FD000900D0020002002400348016941F080018B
:100FE0000161002070470000002002402DE9F05F01
:100FF0000746884615461E460024DFF8749099F887
:101000001800012809D0012089F818004CF2503B43
:101010005846FFF717FC18B126E00220BDE8F09F04
:10102000012F05D0022F05D00427DFF848A019E0D2
:101030000127FAE70227F8E7220128463146FFF7A1
:10104000F0F881B208EB4400FFF7D4FB5846FFF7F5
:10105000F9FBDAF8101021F00101CAF8101018B9E4
:10106000641CE4B2BC42E7D3002189F81810D5E72C
:10107000900D002000200240002006490A69120657
:1010800007D5054A4A60054A4A600969090600D53C
:10109000012070470020024023016745AB89EFCD56
:1010A0002DE9F04F0022DFF8D0904FF001084FF00B
:1010B0000F0C5BE008FA02F4A2460C40002C54D05E
:1010C00022F0030303EB0905AB689607370F0CFA10
:1010D00007F606EA030BB0F1904F04D0274B984275
:1010E00003D1012311E000230FE0254B984201D1E9
:1010F00002230AE0234B984201D1032305E0224B4F
:10110000984201D1042300E00523BB405B4512D186
:101110001E4F3B68A3433B603F1D3B68A3433B60BE
:101120003F1D3B68A3433B603B1D1F68A7431F60F7
:10113000AB68B343AB60046855000323AB409C43EA
:101140000460D40800EB8404266A5507EF0E0CFAFD
:1011500007F5AE432662C4689C43C460446824EA31
:101160000A04446084689C438460521C31FA02F390
:10117000A0D1BDE8F08F000000000140000400484D
:1011800000080048000C004800100048000401401E
:101190002DE9F84F0022DFF880914FF0010809F1A6
:1011A000040A03274FF00F0C0AF1040BACE008FA15
:1011B00002F52B40002B72D00C7904F00304012CB3
:1011C00001D0022C15D18668540007FA04FE26EAE5
:1011D0000E06D1F80CE00EFA04FE4EEA060EC0F838
:1011E00008E04468AC430D79C5F3001595402543EC
:1011F00045600C79E443A40708D0C568540007FA99
:1012000004F6B5438E68A6402E43C6600C7904F000
:101210000304022C11D1D40800EB8406356A54076C
:10122000E40E0CFA04FE25EA0E05D1F810E00EFAE1
:1012300004FE4EEA050EC6F820E00568540007FAE1
:1012400004F6B5430E7906F00306A6402E43066069
:101250004C6814F4403F56D0304CA56945F0010568
:10126000A561A46904F0010400942D4C22F003054B
:101270002E19B56894074FEA147E0CFA0EF4A543B4
:10128000B0F1904F04D0274CA04203D1012412E0CA
:10129000002410E0244CA04202D102240BE032E0F2
:1012A000224CA04201D1032405E0214CA04201D1EF
:1012B000042400E0052404FA0EF42C43B460D9F8A9
:1012C00000409C434D68ED0300D51C43C9F8004025
:1012D000DAF800409C434D68AD0300D51C43CAF8C2
:1012E0000040DBF800409C434D68ED0200D51C43F4
:1012F000CBF80040084D0C352C689C434E68B60274
:1013000000D51C432C60521C0B6833FA02F47FF4A6
:101310004EAFBDE8F88F000000040140001002400D
:10132000000001400004004800080048000C00488C
:1013300000100048002A01D0816170478162704727
:10134000014880687047000054000020024881680E
:1013500002781144816070475400002010B507489E
:10136000016841F010010160032000F07FF80020C7
:1013700000F006F800F026F8002010BD0020024022
:1013800070B504460D4D4FF47A712878B1FBF0F03A
:101390000B490968B1FBF0F000F0B1FC08B1012085
:1013A00070BD102C07D200222146501E00F03EF8DE
:1013B0006C60002070BD012070BD00005400002052
:1013C0006000002008B50948816941F00101816190
:1013D000816901F001010091C16941F08051C16151
:1013E000C06900F08050009008BD0000001002406D
:1013F00000280DDB00F01F02012191404009800010
:1014000000F1E020C0F88011BFF34F8FBFF36F8F62
:101410007047002809DB00F01F02012191404009BC
:10142000800000F1E020C0F800117047F0B40D46D4
:101430000D4B1B68C3F30223C3F10704042C00D92E
:101440000424191D072901D2002300E0DB1E012618
:1014500006FA04F1491E294099409E40761E164026
:101460003143F0BC00F08EBD0CED00E000F0070150
:10147000054A10684FF6FF03184040EA012003496F
:1014800008431060704700000CED00E00000FA0512
:10149000BFF34F8F05480168054A01F4E06111432D
:1014A0000160BFF34F8F00BFFDE700000CED00E0CF
:1014B0000400FA052DE9F04704460D46002C17D02C
:1014C000DFF89481D8F8000000F00700A84211D29C
:1014D000D8F8000020F007002843C8F80000D8F82A
:1014E000000000F00700A84204D00120BDE8F0870A
:1014F0000120FBE72078594E800705D57068A16868
:1015000020F0F000084370602078C00765D0606864
:10151000012201280CD0022822D0022393FAA3F141
:10152000B1FA81F141F02001490931D0316830E050
:101530004FF4003393FAA3F1B1FA81F141F02001A5
:10154000490901D0316800E0716A93FAA3F3B3FA54
:1015500083F303F01F039A40114225D10120C5E710
:101560004FF0007393FAA3F1B1FA81F141F0200139
:10157000490901D0316800E0716A93FAA3F3B3FA24
:1015800083F303F01F039A4011420DD10120ADE710
:10159000716A93FAA3F3B3FA83F303F01F039A403B
:1015A000114201D10120A1E7716821F0030101433B
:1015B0007160FFF7C5FE074641F2883906E0FFF784
:1015C000BFFEC01B484501D903208FE770686168E2
:1015D00000F00C00B0EB810FF1D1D8F8000000F062
:1015E0000700A8420ED9D8F8000020F007002843D1
:1015F000C8F80000D8F8000000F00700A84201D0A9
:10160000012073E72078400705D57068E16820F471
:10161000E060084370602078000706D57068216993
:1016200020F4605040EAC100706000F01FF871685B
:10163000F02292FAA2F201F0F001B2FA82F2D14065
:10164000074A515CC8400749086007480068FFF72F
:1016500097FE00204AE700000020024000100240F0
:10166000DC270008600000205800002010B5164B51
:101670005968164801F00C02042A20D0082A1ED10D
:101680004FF4701494FAA4F401F47012B4FA84F4D0
:10169000E2400F4CA45CDA6A0F2393FAA3F302F042
:1016A0000F02B3FA83F3DA40094B10339A5CC90393
:1016B00006D500231946FEF783FDA0FB040110BDEB
:1016C0000448A4FB000110BD0010024000127A0083
:1016D000BC27000800093D002DE9F84F0446002C06
:1016E00012D02078F84EC0074FF001055ED0706828
:1016F0004FF40038C0F3810001280BD07068C0F3AC
:101700008100022803D01EE00120BDE8F88F706838
:10171000C00318D598FAA8F0B0FA80F040F0200085
:10172000400901D0306800E0706A98FAA8F1B1FA77
:1017300081F101F01F0105FA01F1084275D06068DE
:10174000A0BB0120E1E76068B0F5803F17D0D8B1B9
:10175000B0F5A02F21D0306820F4803030603068A0
:1017600020F480203060F06AA16820F00F00084368
:10177000F0626068C0B3FFF7E3FD07461EE0306823
:1017800040F480303060EEE7306820F48030306024
:10179000306820F480203060E5E7306840F4802035
:1017A0003060306840F480303060DCE73DE0FFF7C7
:1017B000C7FDC01B642801D90320A6E798FAA8F04A
:1017C000B0FA80F040F02000400901D0306800E01D
:1017D000706A98FAA8F1B1FA81F101F01F0105FAD7
:1017E00001F10842E3D020E0FFE7FFF7A9FD07463B
:1017F00006E0FFF7A5FDC01B642801D9032084E79C
:1018000098FAA8F0B0FA80F040F02000400901D02A
:10181000306800E0706A98FAA8F1B1FA81F101F03D
:101820001F0105FA01F10842E3D12078DFF89C821C
:1018300080074FF0000B4FF0020732D570684FF071
:10184000F80A10F00C0F07D07068C0F3810002286E
:1018500028D17068C00325D497FAA7F0B0FA80F0B9
:1018600040F02000400901D0306800E0706A97FA2B
:10187000A7F1B1FA81F101F01F0105FA01F1084267
:1018800004D02069012801D001203EE730689AFA8F
:10189000AAF26169B2FA82F220F0F800914008439E
:1018A00030605CE0206990B395FAA5F0B0FA80F062
:1018B00048F82050FFF744FD814607E0FFF740FD60
:1018C000A0EB0900022801D903201EE797FAA7F030
:1018D000B0FA80F040F02000400901D0306800E00C
:1018E000706A97FAA7F1B1FA81F101F01F0105FAC8
:1018F00001F10842E2D030689AFAAAF26169B2FABC
:1019000082F220F0F80091400843306027E0FFE7C2
:1019100095FAA5F0B0FA80F048F820B0FFF710FD76
:10192000814607E0FFF70CFDA0EB0900022801D972
:101930000320EAE697FAA7F0B0FA80F040F0200022
:10194000400901D0306800E0706A97FAA7F1B1FA57
:1019500081F101F01F0105FA01F10842E2D120787E
:1019600000076DD5A069A8B395FAA5F0B0FA80F08C
:1019700008EB8000C0F88054FFF7E2FC814607E0E6
:10198000FFF7DEFCA0EB0900022801D90320BCE62A
:1019900097FAA7F0B0FA80F040F06000B5EB501F66
:1019A00001D130680BE097FAA7F0B0FA80F040F070
:1019B0006000B7EB501F01D1306A00E0706A97FAFF
:1019C000A7F1B1FA81F101F01F0205FA02F1084214
:1019D000D6D035E0FFE795FAA5F0B0FA80F008EB35
:1019E0008000C0F880B4FFF7ABFC814607E0FFF74A
:1019F000A7FCA0EB0900022801D9032085E697FA8D
:101A0000A7F0B0FA80F040F06000B5EB501F01D1B4
:101A100030680BE097FAA7F0B0FA80F040F0600071
:101A2000B7EB501F01D1306A00E0706A97FAA7F156
:101A3000B1FA81F101F01F0205FA02F10842D6D194
:101A4000207840076ED54FF00009F069C00009D436
:101A5000F06940F08050F061F06900F08050009033
:101A60004FF001091A480168C90513D4016841F40F
:101A700080710160FFF764FC824607E0FFF760FCBD
:101A8000A0EB0A00642801D903203EE61048006854
:101A9000C005F3D5E068012810D0D8B1052822D0C0
:101AA000306A20F001003062306A20F004003062B9
:101AB000E068B0B3FFF744FC824627E0306A40F0AC
:101AC00001003062F4E700000010024000004242D2
:101AD00000700040306A20F001003062306A20F06F
:101AE00004003062E4E7306A40F004003062306A9B
:101AF00040F001003062DBE7FFF722FCA0EB0A01B7
:101B000041F28830814201D90320FEE597FAA7F01F
:101B1000B0FA80F040F04000B5EB501F03D13068C0
:101B20000DE017E04CE097FAA7F0B0FA80F040F033
:101B30004000B7EB501F01D1306A00E0706A97FA9D
:101B4000A7F1B1FA81F101F01F0105FA01F210428B
:101B5000D2D02EE0FFF7F4FB824609E0FFF7F0FB5E
:101B6000A0EB0A0141F28830814201D90320CCE583
:101B700097FAA7F0B0FA80F040F04000B5EB501FA4
:101B800001D130680BE097FAA7F0B0FA80F040F08E
:101B90004000B7EB501F01D1306A00E0706A97FA3D
:101BA000A7F1B1FA81F101F01F0105FA01F210422B
:101BB000D4D1B9F1010F03D1F06920F08050F06168
:101BC000E06980B37168C1F38101022977D04FF0D9
:101BD00080794FF00077022809D099FAA9F0B0FA7D
:101BE00080F048F820B0FFF7ABFB04465DE099FABF
:101BF000A9F0B0FA80F048F820B0FFF7A1FB8246C8
:101C000007E0FFF79DFBA0EB0A00022801D90320A3
:101C10007BE597FAA7F0B0FA80F040F02000400989
:101C200002D0306801E068E0706A97FAA7F1B1FA73
:101C300081F101F01F0105FA01F10842E1D1D4E977
:101C400008100843716821F474110843706099FA10
:101C5000A9F0B0FA80F048F82050FFF771FB044675
:101C600006E0FFF76DFB001B022801D903204CE5BD
:101C700097FAA7F0B0FA80F040F02000400901D0B8
:101C8000316800E0716A97FAA7F0B0FA80F000F0CE
:101C90001F0005FA00F00142E3D02EE0FFF750FBF1
:101CA000001B022801D903202FE597FAA7F0B0FA0C
:101CB00080F040F02000400902D0316801E00BE0E4
:101CC000716A97FAA7F0B0FA80F000F01F0005FAE9
:101CD00000F00142E2D110E001280CD07068226AC5
:101CE00000F48031914204D1616A00F4701088429E
:101CF00003D0012009E5012007E5002005E510B526
:101D0000401EB0F1807F01D3012010BD4FF0E024D0
:101D100060610F21601700F035F90020A0610720F5
:101D20002061002010BD012484F31388FFF7B0FB6D
:101D3000FAE7000001B481B0019800680A49084040
:101D4000B0F1005F03D0012002B0FFF7E1B80198C5
:101D5000406800900549009808600199096881F37E
:101D6000088802B0004700000000FE2F000000209D
:101D700010B5104C0E482060182060600020A06054
:101D8000E0604FF4403121616061A0610121E161B7
:101D900021626062A062E0622046FEF7C3FE08B1E5
:101DA000FEF7A7FC2068016821F48031016010BDB6
:101DB00000640040A4000020F0B587B0142102A800
:101DC000FEF746FA2248416941F4800141614169C8
:101DD00001F480010191416941F40031416141699F
:101DE00001F400310191416941F48021416141696F
:101DF00001F480210191416941F400214161406970
:101E000000F4002001904FF480544FF090470022DE
:101E100021463846FFF78EFA0E4E01220221304647
:101E2000FFF788FA02940125039500240494059491
:101E300002A93846FFF7ACF90220029003950494FA
:101E4000059402A93046FFF7A3F907B0F0BD0000E2
:101E50000010024000080048FEE77047704700008D
:101E600003488188491C81804188491C4180704712
:101E700004000020704710B5FFF7F2FFBDE81040E6
:101E8000FFF764BA30B58FB0282105A8FEF7E0F956
:101E900014216846FEF7DCF9092005904FF48031E3
:101EA000069100240794012009900B9002250C95BF
:101EB0000D914FF4E0100E9005A8FFF70DFC08B14E
:101EC000FEF717FC0F200090019502944FF48060FC
:101ED0000390049402216846FFF7ECFA002801D031
:101EE000FEF707FC0FB030BD0248016841F47001F5
:101EF0000160704788ED00E00148FEF763BD000017
:101F0000A4000020FEE700000F4D104E104C0DE025
:101F1000002202212846FFF70DFA3220FEF7F8FFD3
:101F20000C48FEF737FD3046FFF704FF0A48FEF77E
:101F300089FA00F0A5F900F0D7F900F0B9F9617855
:101F40000129F3D1E4E70000000800480030000850
:101F5000E4000020A40000204400002010B5FEF79B
:101F6000EFFB064900208870C8800870487008742C
:101F700003494FF47A728A80488010BDE400002043
:101F8000040000200907090E002804DB00F1E0200E
:101F900080F80014704700F00F0000F1E02080F896
:101FA000141D704702E008C8121F08C1002AFAD1A8
:101FB00070477047002001E001C1121F002AFBD1C9
:101FC0007047000010B5184B04891A688C4215D36D
:101FD000546924F0020454610289521A02811A6879
:101FE000536943F002035361C288114489B24288A5
:101FF0008A4201D8891A89B2C18010BD516921F085
:102000000201516102890021018119684B6943F085
:1020100002034B61C188114489B242888A4201D8C7
:10202000891A89B2C18010BDA400002002898A42A9
:1020300008D3C288114489B242888A4203D8891AD7
:1020400089B200E00021C068405C7047FFF786F964
:10205000FFF718FFFFF7B0FEFFF78AFEFFF77EFFDE
:10206000FFF752FFFEE7000070B50B212448FEF792
:10207000F3FA234D010EE972010C2973010A697309
:10208000A873214C1F48216B00880860216B002039
:10209000C860216B8860216B08200861216B28785B
:1020A0000875216B6878487502202918236B8A7897
:1020B00000F114015A54401CC0B20828F5D3142171
:1020C0001148FEF74BFE012801D1FFF751FE216BAD
:1020D0000620086100202918236B8A7A00F1140178
:1020E0005A54401CC0B20628F5D314210648FEF706
:1020F00035FE012803D1BDE87040FFF739BE70BD41
:102100002200002044000020A400002070B511210E
:102110002C48FEF7A1FA2B4C010E6174010CA1743E
:10212000010AE1742075294D2748296B0088086051
:10213000286B08260661296B20780875296B607862
:102140004875022021182B6B8A7800F114015A542B
:10215000401CC0B20828F5D314211C48FEF7FEFD30
:10216000012801D1FFF704FE286B06610020211829
:102170002B6B8A7A00F114015A54401CC0B2082813
:10218000F5D314211148FEF7E9FD012801D1FFF72D
:10219000EFFD296B04200861002021182B6B8A7C3D
:1021A00000F114015A54401CC0B20428F5D3142184
:1021B0000648FEF7D3FD012803D1BDE87040FFF7C4
:1021C000D7BD70BD0C00002044000020A4000020FA
:1021D00070B5284C020AA271E0712172080A60727F
:1021E0000A212046FEF738FA010EA172010CE172B5
:1021F000010A21736073204D0020296BC860296B90
:1022000088601E48296B00880860296B08200861D7
:10221000296B20780875296B607848750220211891
:102220002B6B8A7800F114015A54401CC0B2082864
:10223000F5D314211048FEF791FD012801D1FFF7D5
:1022400097FD296B05200861002021182B6B8A7AE5
:1022500000F114015A54401CC0B20528F5D31421D2
:102260000548FEF77BFD012803D1BDE87040FFF76C
:102270007FBD70BD32000020A4000020440000207B
:102280000949887800280ED1087C042809D2074A19
:102290009388322B07D300239380401C0874FFF7E8
:1022A00035BF012048707047E40000200400002082
:1022B00010B50B4C6078002811D1A07800280ED002
:1022C000084840F6B8324188914208D9002141803F
:1022D000E1884CF20230FFF77BFF0120607010BDF7
:1022E000E4000020040000202DE9F047304C0127D5
:1022F000002620782F4D01281ED126702846A97867
:102300008088012906D0022908D003290AD005298E
:1023100012D10CE00021FFF75BFF0DE0E988FFF729
:1023200057FF09E00021FFF753FF6F7004E0FFF74C
:102330009BFEAE706E702E74287801282FD12E70FF
:10234000E9884CF202694A1EB2F5806F29D2DFF8A3
:10235000648008F1130811F8080048B14CF202201B
:10236000FFF736FF4846BDE8F047E121FFF730BFF1
:102370001148A96800EBC2102022FEF7EDF948B120
:102380004FF47A74EE214846FFF722FF2046FEF70D
:10239000BFFDF7E7E88800F8087027706680BDE8A1
:1023A000F0874846BDE8F047E221FFF711BF000083
:1023B00004000020E40000200030000800000000BD
:1023C000B71DC1046E3B8209D926430DDC76041388
:1023D0006B6BC517B24D861A0550471EB8ED08261F
:1023E0000FF0C922D6D68A2F61CB4B2B649B0C35BC
:1023F000D386CD310AA08E3CBDBD4F3870DB114C69
:10240000C7C6D0481EE09345A9FD5241ACAD155F4B
:102410001BB0D45BC2969756758B5652C836196A54
:102420007F2BD86EA60D9B6311105A6714401D793F
:10243000A35DDC7D7A7B9F70CD665E74E0B62398E9
:1024400057ABE29C8E8DA191399060953CC0278B53
:102450008BDDE68F52FBA582E5E66486585B2BBEDA
:10246000EF46EABA3660A9B7817D68B3842D2FADF7
:102470003330EEA9EA16ADA45D0B6CA0906D32D49A
:102480002770F3D0FE56B0DD494B71D94C1B36C7CF
:10249000FB06F7C32220B4CE953D75CA28803AF2D8
:1024A0009F9DFBF646BBB8FBF1A679FFF4F63EE133
:1024B00043EBFFE59ACDBCE82DD07DEC77708634F8
:1024C000C06D4730194B043DAE56C539AB06822767
:1024D0001C1B4323C53D002E7220C12ACF9D8E12A6
:1024E00078804F16A1A60C1B16BBCD1F13EB8A01DB
:1024F000A4F64B057DD00808CACDC90C07AB977868
:10250000B0B6567C69901571DE8DD475DBDD936BAA
:102510006CC0526FB5E6116202FBD066BF469F5E8B
:10252000085B5E5AD17D1D576660DC5363309B4D5E
:10253000D42D5A490D0B1944BA16D84097C6A5ACEC
:1025400020DB64A8F9FD27A54EE0E6A14BB0A1BFB2
:10255000FCAD60BB258B23B69296E2B22F2BAD8AE1
:1025600098366C8E41102F83F60DEE87F35DA99996
:102570004440689D9D662B902A7BEA94E71DB4E059
:10258000500075E4892636E93E3BF7ED3B6BB0F32E
:102590008C7671F7555032FAE24DF3FE5FF0BCC60F
:1025A000E8ED7DC231CB3ECF86D6FFCB8386B8D552
:1025B000349B79D1EDBD3ADC5AA0FBD8EEE00C6932
:1025C00059FDCD6D80DB8E6037C64F643296087A38
:1025D000858BC97E5CAD8A73EBB04B77560D044F8B
:1025E000E110C54B383686468F2B47428A7B005C0C
:1025F0003D66C158E4408255535D43519E3B1D25C5
:102600002926DC21F0009F2C471D5E28424D1936FB
:10261000F550D8322C769B3F9B6B5A3B26D6150340
:1026200091CBD40748ED970AFFF0560EFAA011108F
:102630004DBDD014949B93192386521D0E562FF135
:10264000B94BEEF5606DADF8D7706CFCD2202BE283
:10265000653DEAE6BC1BA9EB0B0668EFB6BB27D7C6
:1026600001A6E6D3D880A5DE6F9D64DA6ACD23C4C7
:10267000DDD0E2C004F6A1CDB3EB60C97E8D3EBDD6
:10268000C990FFB910B6BCB4A7AB7DB0A2FB3AAEFF
:1026900015E6FBAACCC0B8A77BDD79A3C660369B44
:1026A000717DF79FA85BB4921F4675961A16328803
:1026B000AD0BF38C742DB081C330718599908A5D18
:1026C0002E8D4B59F7AB085440B6C95045E68E4E97
:1026D000F2FB4F4A2BDD0C479CC0CD43217D827B12
:1026E0009660437F4F460072F85BC176FD0B8668AB
:1026F0004A16476C93300461242DC565E94B9B1144
:102700005E565A1587701918306DD81C353D9F02DA
:1027100082205E065B061D0BEC1BDC0F51A6933777
:10272000E6BB52333F9D113E8880D03A8DD097242E
:102730003ACD5620E3EB152D54F6D4297926A9C5B8
:10274000CE3B68C1171D2BCCA000EAC8A550ADD662
:10275000124D6CD2CB6B2FDF7C76EEDBC1CBA1E3CD
:1027600076D660E7AFF023EA18EDE2EE1DBDA5F0E6
:10277000AAA064F4738627F9C49BE6FD09FDB88915
:10278000BEE0798D67C63A80D0DBFB84D58BBC9ADE
:1027900062967D9EBBB03E930CADFF97B110B0AF7B
:1027A000060D71ABDF2B32A66836F3A26D66B4BCA2
:1027B000DA7B75B8035D36B5B440F7B102030405A2
:1027C000060708090A0B0C0D0E0F10100102030476
:1027D00005060708090A0B0C0D0E0F10000000007B
:1027E0000000000001020304060708090C28000885
:1027F0000000002064000000A41F000870280008EA
:10280000640000204C1D0000B41F00080000000000
:10281000000000000000000055AA07150C0BC109BC
:102820004D432056312E322E3200000000F055AAC2
:1028300007150C05A90341434B00000000F055AA01
:1028400007150C040000000000000000F00000006C
:102850001507000800000000000000008A050020A5
:1028600001000000100000000000000000127A00CB
:040000050800018965
:00000001FF
